:10000000B8200020290B0000250B0000250B000064
:1000100000000000000000000000000000000000E0
:10002000000000000000000000000000250B0000A0
:100030000000000000000000250B0000250B000060
:10004000250B0000250B0000250B0000250B0000F0
:10005000A1040000250B0000250B0000250B00006B
:10006000250B0000F903000009040000190400003A
:100070002904000039040000490400003503000091
:100080004503000055030000250B0000250B000070
:10009000250B0000250B0000250B0000350100009A
:1000A000250B0000250B0000250B0000250B000090
:1000B0000000000010B5064C2378002B07D1054B3B
:1000C000002B02D0044800E000BF0123237010BDC4
:1000D0000C00002000000000D00D0000084B10B5FF
:1000E000002B03D00749084800E000BF0748036819
:1000F000002B00D110BD064B002BFBD09847F9E731
:100100000000000010000020D00D0000D00D000005
:100110000000000003685A7E52B2002AFBDB022274
:10012000197B0A431A730268537E5BB2002BFBDB18
:100130007047000070B5284B1C6823681A7EDD7D6F
:1001400015400122154228D01A7621684B7E5BB2F9
:10015000002BFBDB6269931C63614B8B9BB21380AA
:10016000238B013B9BB22383002B10D101222168FA
:100170008A75217F052910D12377E37E13420CD0A5
:10018000A37E134209D02000A368984705E0637F4F
:10019000002B02D02000114B984704231D420BD0A6
:1001A00022681376E27E023B1A4205D0A27E1A42F2
:1001B00002D02000E368984702231D420BD022683A
:1001C0001376E27EDB181A4205D0A27E1A4202D0D4
:1001D00023692000984770BD6000002015010000D1
:1001E000014B5878C009704700180040022310B531
:1001F000044A11780B431370034B98470028FBD136
:1002000010BDC04600180040E1010000402307B5C2
:10021000104A052091690B439361002301A90B70DB
:100220000D4B98470D4B0520984701230C4A117838
:100230000B4313700B4B98470028FBD102000A4B6D
:100240001A5004304028FBD11022084B1A60084B8A
:10025000984707BD00040040F50900006D09000043
:1002600000180040E10100006400002000E100E00F
:10027000ED0100000023012203604360837202331A
:1002800002724272C3727047F7B50C0000262379E0
:1002900001A94E70CE700B70237A05008B70207808
:1002A000134B984733001F2D00D8124B0721A27A19
:1002B00029408900E67A002A01D0082216430F2738
:1002C0008E408F403100EA0892009A189069B84336
:1002D00001439161617A0122002904D0AA40596941
:1002E0000A435A61F7BDAA40596991435961F9E738
:1002F000C90A000000180040F8B500250B4B80002B
:10030000C4582368626BDE6AA36B13401E40084B1F
:10031000EF58374205D063195B682000984723687F
:10032000DF620435302DF2D1F8BDC046A4000020B4
:10033000800D000010B50020014B984710BDC0464D
:10034000F902000010B50120014B984710BDC046CE
:10035000F902000010B50220014B984710BDC046BD
:10036000F902000070470000F0B5060085B001AC4E
:1003700020000A4B0D001700984700230196012624
:100380006360237221002800054BE6729847320013
:1003900029003800034B984705B0F0BD75020000F6
:1003A0008902000059040000704770470A2110B507
:1003B00008000B4C0B4AA0470B210B4A0800A04732
:1003C0000C210A4A0800A047094C01210A20A04735
:1003D00001210B20A04701210C20A04710BDC046E1
:1003E00069030000AB030000A903000065030000DF
:1003F000810400007047000010B5024B00201B680C
:10040000984710BD2800002010B5024B01205B6802
:10041000984710BD2800002010B5024B02209B68B1
:10042000984710BD2800002010B5024B0320DB6860
:10043000984710BD2800002010B5024B04201B690E
:10044000984710BD2800002010B5024B05205B69BD
:10045000984710BD2800002010B51723002A06D1A8
:10046000064B8900CC58002C03D1C850230018003B
:1004700010BD13008442FAD01D23F8E76400002069
:100480001723002906D11F2806D8163B8340034AAC
:10049000D3600B0018007047C960FFDE00180040F1
:1004A000002370B501250B4C237023780F2B00D946
:1004B00070BD29009940084A1069084206D01161B0
:1004C000064A9B009B58002B00D0984723780133A5
:1004D0002370EAE7B000002000180040640000200C
:1004E00070B5094B00209847FA21084C8900050097
:1004F000A047074B074918602800A0470522064B74
:100500001860064B1A6070BDE5080000210C000061
:100510000000002040420F000400002010E000E036
:10052000094B196800290BD1EFF31080074A002806
:1005300005D172B6BFF35F8F0549087001211170B4
:100540001A6801321A607047400000204400002001
:1005500008000020084B1A68013A1A601B68002B3B
:1005600009D1064B1B78002B05D00122044B1A70D1
:10057000BFF35F8F62B67047400000204400002048
:1005800008000020F7B50125002701AC084E210026
:100590003E206570A7702570B0478022054BD205BC
:1005A0001A6021000F2027706570B047F7BDC04664
:1005B000B90500009844004107B5802201AB1A70CC
:1005C0000A785A704A789A708A781900DA70014B62
:1005D000984707BDC90A000010230249CA681A4299
:1005E000FCD070470008004070B5082806D800F01D
:1005F0000DFB0805053030120B15280000242000E3
:1006000070BD164B1C69FAE7154B164C1B6A9B050F
:100610009B0FDC40F3E7114B5C69F0E70F4D0024C2
:100620002B689B07EBD5104B984724222B6813406F
:10063000042B11D120000D4B9847AC68A4B2444361
:10064000DDE70B4B00241B785B07D8D5034BDC6838
:10065000D5E780242402D2E7064CD0E748000020EA
:100660000008004000127A00D9050000110A0000BD
:1006700050080040006CDC0270B584780278457840
:10068000012040260540204080240849AD010B6A26
:10069000C001B3432B43A343034303200240044858
:1006A0001202034013430B6270BDC04600080040B5
:1006B000FFFCFFFFF8B5082806D800F0A7FA1405DC
:1006C000050C0E1A072034001720F8BD0223194A22
:1006D000116A0B4313620020F7E70223154A916960
:1006E0000B439361F7E70223124A118A0B431382EB
:1006F000F1E702230F4A918A0B439382EBE7022230
:1007000000240D4E0B4D33680C4F13433360AA8405
:10071000B847B368EB627368AB62AC84B8473368C0
:100720009BB2AB84D7E70223054A11780B431370C1
:10073000D1E7C0460008004048000020D90500006D
:10074000440800407FB5C2221E21194BD2009A6096
:10075000184A0024536801AD8B43536001232B706A
:10076000E0B22900144B01349847252CF8D100241D
:100770006B4601265C709E701C7068460F4B984754
:100780000F4B062098470F4B98470F4B29001C72C0
:100790005C729C72DC72062320002B700B4B6E6027
:1007A0006C702C726C7298472000094B98477FBD83
:1007B0000008004000400041F509000079060000F3
:1007C000B5060000E1070000000400400108000039
:1007D000A5080000014B5878C0097047000C004084
:1007E0000823054A91690B4393610123034A13705F
:1007F00011781942FCD1704700040040000C004001
:10080000F8B50C784B782402060005000443002B51
:1008100002D08023DB021C434B7A002B02D08023C2
:100820001B031C434B68012B12D95D1E1D40022285
:10083000002D06D01D02802335439B0207E00135C1
:1008400052009A42FBD380232D0235435B031C43A5
:100850000B7A002B02D080239B031C430C4FB8471C
:100860000028FBD10B4B98470B4B1E70B847002854
:10087000FCD10A4B9D601D00B8470028FCD18022A6
:100880006B68520213401C436C60054B9847F8BDDF
:10089000D507000021050000080C0040000C0040B6
:1008A0005505000070B50500094CA0470028FBD194
:1008B000084B9847084B1D70A0470028FCD18023A7
:1008C000064A5B0251680B435360054B984770BD65
:1008D000D507000021050000040C0040000C00407A
:1008E00055050000F7B50700184EB0470028FBD1AA
:1008F000174B9847174B1F700193B0470028FCD146
:10090000154D164B6868C004C00E98470400019B43
:100910001F706B68DB02DB0F0193114B1F70B04738
:100920000028FCD1AD680F4B9847019B2D022D0C80
:10093000002B08D1012D04D9200029000A4B98472B
:1009400004002000FEBD0135EC40FAE7D5070000A9
:1009500021050000040C0040000C0040E9050000E7
:10096000080C004055050000210C000010B50400E3
:10097000064B9847064B074A1C7080235188DB01C1
:100980000B435380044B984710BDC046210500001F
:10099000020C0040000C00405505000010B504009A
:1009A0000E4B98470E4B0F4A1C700F4B0F4C58883C
:1009B00059880005114059805988000F21405980FD
:1009C00011008022D2015C881442FCD15A880002B6
:1009D0000A4002435A80064B984710BD210500008B
:1009E000020C0040FFF0FFFF000C0040FFBFFFFFC4
:1009F0005505000010B50C78034B240204439847BA
:100A0000024BA4B25C8010BD9D090000000C0040A8
:100A100010B50400064B9847064B1C70064B5C88CB
:100A2000064B2405240F98472000054B984710BD1E
:100A300021050000020C0040000C0040550500009C
:100A4000E5080000D37830B5002B35D11478802C20
:100A500003D0802324065B02234302255478AC4351
:100A600006D19478002C24D18024A4022343416031
:100A70005478013C012C01D8124C2340A0248DB2A3
:100A8000E4052C431C438462D0240D0C24062C4323
:100A90001C438462D478002C0AD15B0303D593787D
:100AA000012B0CD181615378013B012B00D881606F
:100AB00030BDC024E402D9E741600023DEE7416194
:100AC000F1E7C046FFFFFBFF10B503000A00440931
:100AD000C1090020814202D10449E00140181F21D0
:100AE0000B401E399940024B984710BD004400410D
:100AF000450A00007047000010B5054B9847054BAC
:100B00009847054B9847054B9847054B984710BDAC
:100B10004507000085050000F50A00000D020000F1
:100B2000F50A0000FEE700002148224970B588421E
:100B300004D00023204CCA18A24232D300211F4BFC
:100B40001F4A934231D3FF211E4B1F4A8B439360B0
:100B500002220C25082430261C4B1D485A62C378FB
:100B6000FC398B431343C370C378AB432343C37037
:100B7000184B987BB0430600202030439873987B35
:100B8000A84304439C73987B884302439A73802351
:100B9000114A51680B435360104B9847104B9847CC
:100BA000FEE7C55804331560C5E702C3C9E7C04670
:100BB000D00D0000000000200C0000200C000020E0
:100BC000B40000200000000000ED00E0FC700041D7
:100BD000005000410048004100400041390D000034
:100BE000E50B000010B5054B9847054B9847054BA2
:100BF0009847054B9847002010BDC046F90A0000F1
:100C0000E1040000F5030000AD03000002B47146EA
:100C100049084900095C49008E4402BC7047C0463F
:100C2000002243088B4274D303098B425FD3030A2B
:100C30008B4244D3030B8B4228D3030C8B420DD33E
:100C4000FF22090212BA030C8B4202D312120902CC
:100C500065D0030B8B4219D300E0090AC30B8B420A
:100C600001D3CB03C01A5241830B8B4201D38B03B8
:100C7000C01A5241430B8B4201D34B03C01A52415D
:100C8000030B8B4201D30B03C01A5241C30A8B42A0
:100C900001D3CB02C01A5241830A8B4201D38B028B
:100CA000C01A5241430A8B4201D34B02C01A52412F
:100CB000030A8B4201D30B02C01A5241CDD2C309A1
:100CC0008B4201D3CB01C01A524183098B4201D31D
:100CD0008B01C01A524143098B4201D34B01C01A08
:100CE000524103098B4201D30B01C01A5241C30880
:100CF0008B4201D3CB00C01A524183088B4201D3EF
:100D00008B00C01A524143088B4201D34B00C01ADA
:100D10005241411A00D20146524110467047FFE746
:100D200001B5002000F006F802BDC0460029F7D04A
:100D300076E770477047C04670B500260C4D0D4CE5
:100D4000641BA410A64209D1002600F031F80A4D18
:100D50000A4C641BA410A64205D170BDB300EB5829
:100D600098470136EEE7B300EB5898470136F2E7B3
:100D7000BC0D0000BC0D0000BC0D0000C00D00004B
:100D80000100000002000000040000000800000054
:100D90000010000000200000004000000080000063
:100DA0000000010000000200000004000000080034
:100DB000F8B5C046F8BC08BC9E467047DD00000090
:100DC000F8B5C046F8BC08BC9E467047B5000000A8
:0C0DD000401F00000800000001000000AF
:0400000300000B29C5
:00000001FF
